:100000000C94F6000C9413010C9413010C9413013E
:100010000C9413010C9413010C9413010C94130110
:100020000C9413010C9439060C9413010C940007E2
:100030000C9413010C943C070C9413010C941301C1
:100040000C9413010C9413010C9413010C94820270
:100050000C941301C204CC04C504CC04C804CC0421
:10006000CA04CC041606160616061606160616064A
:10007000CE04E604D304E604D804E604DD04E60472
:100080001606160616061606160616061606160690
:10009000E904EE04F304F804FD04020507050C0569
:1000A0001606160616061606160616061606160670
:1000B000110516051B05200525052A052F05350503
:1000C0003A054B0554055D05600575057E058705F8
:1000D0008A0593059C05A505AE05B705C005C905AC
:1000E000D205DB05E705F405160616061606160604
:1000F0001606160616061606160616061606160620
:10010000160616061606160616061606160616060F
:1001100016061606160616061606160616061606FF
:1001200016061606160616061606160616061606EF
:1001300016061606160616061606160616061606DF
:1001400016061606160616061606160616061606CF
:1001500016061606160616061606160616061606BF
:1001600016061606160616061606160616061606AF
:10017000160616061606160616061606160616069F
:10018000160616061606160616061606160616068F
:10019000FD05020607060C06110605A84CCDB2D4D3
:1001A0004EB93836A9020C50B9918688083CA6AAE7
:1001B000AA2ABE000000803F493243205374617474
:1001C000653A20307825780D0A000D0A5374617263
:1001D000740D0A0045464765666700202B2D2E30BA
:1001E00031323334353637383968000011241FBEB8
:1001F000CFE5D8E0DEBFCDBF10E0A0E6B0E0E6E599
:10020000FEE202C005900D92A037B107D9F721E0B8
:10021000A0E7B0E001C01D92AC36B207E1F70E9442
:1002200032080C9429170C9400008091A300807F61
:100230008093A30090B326B33091A3009074892FCC
:1002400090E043E0959587954A95E1F72770822BDA
:10025000809590958F709927832B8093A300809130
:10026000EA009091EB00209166003091670028171A
:10027000390709F449C08091EA009091EB00892B7D
:1002800031F485B3837F85BB8FB58F7729C080918B
:10029000EA009091EB008115904819F485B38C60C9
:1002A0001CC080916900811107C08091EA00909183
:1002B000EB001816190654F080916900882351F05C
:1002C0008091EA009091EB0097FF04C085B3877F8F
:1002D000846003C085B38B7F886085BB8FB58068E1
:1002E0008FBD8091EA009091EB009093670080931E
:1002F00066008091EA009091EB0097FF03C0919512
:10030000819591099BBD8ABD8091E8009091E9009B
:1003100020916400309165002817390709F449C01D
:100320008091E8009091E900892B31F485B38F7CAE
:1003300085BB8FB58F7D29C08091E8009091E90041
:100340008115904819F485B380631CC080916800C2
:10035000811107C08091E8009091E90018161906F4
:1003600054F080916800882351F08091E8009091CA
:10037000E90097FF04C085B38F7D806103C085B31A
:100380008F7E806285BB8FB580628FBD8091E800D3
:100390009091E90090936500809364008091E8005B
:1003A0009091E90097FF03C091958195910999BDBE
:1003B00088BD8091E6009091E70020916200309125
:1003C00063002817390709F448C08091E60090912E
:1003D000E700892B31F485B38F7385BB85B58F7D9D
:1003E00029C08091E6009091E7008115904819F4AA
:1003F00085B3806C1CC08091D700811107C08091AB
:10040000E6009091E7001816190654F08091D70085
:10041000882351F08091E6009091E70097FF04C097
:1004200085B38F77806403C085B38F7B806885BB7D
:1004300085B5806285BD8091E6009091E70090933C
:100440006300809362008091E6009091E70097FF3F
:1004500003C091958195910983BD8091E4009091AD
:10046000E50020916000309161002817390709F4F8
:1004700048C08091E4009091E500892B31F482B36B
:10048000837F82BB83B78F7D29C08091E4009091E8
:10049000E5008115904819F482B38C601CC08091EE
:1004A000D600811107C08091E4009091E5001816F4
:1004B000190654F08091D600882351F08091E40011
:1004C0009091E50097FF04C082B3877F846003C0EA
:1004D00082B38B7F886082BB83B7806283BF809149
:1004E000E4009091E500909361008093600080911A
:1004F000E4009091E50097FF03C0919581959109E3
:100500008CBF08951F920F920FB60F9211242F9354
:100510003F934F935F936F937F938F939F93AF938B
:10052000BF93EF93FF9381B1887F8093A10081B146
:10053000887F803A09F483C328F4803669F08038D4
:1005400081F07FC3883B09F40FC2883F09F47BC365
:10055000883A09F076C308C285EC86BF1092ED0098
:1005600072C38091ED008C3209F472C108F05FC053
:10057000813209F4FFC068F5843009F4E3C060F407
:10058000813009F40FC108F4C8C0823009F4CEC02C
:10059000833009F407C1E0C1873009F403C190F446
:1005A000853009F4FFC0863009F0D6C183B12091AF
:1005B0009E0090E0922B9093E7008093E6001092CB
:1005C000D900C8C1883009F4C9C0803209F4EAC032
:1005D000C3C1863209F4E6C0C0F4833209F4D7C03F
:1005E00008F4E0C0843209F4DDC0853209F0B4C1FA
:1005F00083B120919E0090E0922B9093D100809344
:10060000D00081E08093D900A5C1893209F4DBC014
:1006100038F4873209F4CAC0883209F419C19CC180
:100620008A3209F4D0C08B3209F4E4C095C1873511
:1006300009F42FC108F040C0813509F4C4C060F44A
:100640008E3209F4C0C008F4BEC08F3209F4D2C0A3
:10065000803509F4FDC080C1843509F4FEC028F559
:10066000823509F4B0C0833509F076C123B1809199
:100670009A0090919B00A0919C00B0919D00BA2F90
:10068000A92F982F8827822B80939A0090939B0004
:10069000A0939C00B0939D008093EE009093EF0098
:1006A000A093F000B093F10055C1853509F4DAC08C
:1006B000863509F4D7C050C1843909F416C1A8F4AD
:1006C000813909F40AC138F4803909F045C183B190
:1006D000809369003FC1823909F403C1833909F06D
:1006E0003BC183B18093D60035C1803B09F408C17A
:1006F00050F4853909F4FDC0843A09F02DC183B165
:1007000080939F0027C1813B09F401C18F3F09F00D
:1007100023C183B18093EC001FC183B18093ED00AE
:100720008091ED0081508093ED0014C183B1209140
:100730009E0090E0922B9093EB008093EA00109241
:10074000DB0008C183B120919E0090E0922B909332
:10075000E9008093E8001092DA00FCC083B1209198
:100760009E0090E0922B9093E5008093E40010921D
:10077000D800F0C083B120919E0090E0922B90931E
:10078000D5008093D40081E08093DB00E3C083B187
:1007900020919E0090E0922B9093D3008093D20002
:1007A00081E053C083B180939E00D4C083B1209177
:1007B0009E0090E0922B9093CF008093CE0081E03A
:1007C0008093D800C7C023B180919A0090919B007C
:1007D000A0919C00B0919D00BA2FA92F982F882737
:1007E000822B80939A0090939B00A0939C00B093DF
:1007F0009D00B0C023B180919A0090919B00A09180
:100800009C00B0919D00BA2FA92F982F8827BC017A
:10081000CD01622B60939A0070939B0080939C00A3
:1008200090939D0020E038E24EEA55E40E946A135E
:100830000E943E127093D5006093D4007093D30051
:100840006093D20081E08093DB008093DA0082C065
:1008500083B190E0A0E0B0E0C4CF83B190E0A0E02D
:10086000B0E00EC023B18091960090919700A091C6
:100870009800B0919900BA2FA92F982F8827822B22
:100880008093960090939700A0939800B09399005E
:1008900061C023B18091960090919700A09198003B
:1008A000B0919900BA2FA92F982F8827822B809377
:1008B000960090939700A0939800B093990080932E
:1008C000F2009093F300A093F400B093F50081E060
:1008D0008093F6001092A2003DC083B1809368001F
:1008E00039C083B18093D70035C083B18093A50010
:1008F00003C083B18093A40081E08093F6002AC0F6
:1009000083B190E0909395008093940023C083B1CD
:1009100060E070E070919400682B70939500609394
:1009200094006115710579F08CE496E20E94281418
:100930006093C3001092C40089B7816089BF8FEFB4
:100940008093A20007C089B78E7F89BF1092E5000F
:100950001092E40085EC01C085E886BF8091ED002F
:100960008F3F09F066C16FC1E091ED008E2F90E0DE
:10097000FC013297E33AF10508F058C1E65DFF4FFC
:100980000C945B148AB59BB53FC188B599B53CC141
:1009900083B53AC18CB738C113B837C18091E20032
:1009A0009091E3000EC08091E0009091E10009C0B9
:1009B0008091DE009091DF0004C08091DC00909176
:1009C000DD0090939500809394004DC08091940039
:1009D0001BC18091D4009091D50045C08091D40076
:1009E0009091D50011C18091D2009091D3003BC06D
:1009F0008091D2009091D30007C18091D000909156
:100A0000D10031C08091D0009091D100FDC0809183
:100A1000CE009091CF0027C08091CE009091CF0062
:100A2000F3C08091C1009091C2001DC08091C100AF
:100A30009091C200E9C08091BF009091C00013C0A6
:100A40008091BF009091C000DFC08091BD00909167
:100A5000BE0009C08091BD009091BE00D5C08091BC
:100A6000BB009091BC0093B9D0C08091BB00909125
:100A7000BC00CAC08091AB009091AC00A091AD00C9
:100A8000B091AE0080939A0090939B00A0939C003D
:100A9000B0939D0025C080919A0090919B00A091F9
:100AA0009C00B0919D008FC080919A0090919B0016
:100AB000A0919C00B0919D0092C080919A00A4C02A
:100AC0008091A7009091A800A091A900B091AA00E0
:100AD0008093960090939700A0939800B09399000C
:100AE0008B2F9927AA27BB278FC0809196009091C2
:100AF0009700A0919800B091990065C080919600F0
:100B000090919700A0919800B091990068C0809151
:100B100096007AC08091B7009091B800A091B9007A
:100B2000B091BA00DDCF8091B7009091B800A0914C
:100B3000B900B091BA0047C08091B7009091B80059
:100B4000A091B900B091BA004AC08091B7009091CD
:100B5000B800A091B900B091BA0056C08091B3001E
:100B60009091B400A091B500B091B600B9CF80913A
:100B7000B3009091B400A091B500B091B60023C02D
:100B80008091B3009091B400A091B500B091B600EF
:100B900026C08091B3009091B400A091B500B091AF
:100BA000B60032C08091AF009091B000A091B1002A
:100BB000B091B20095CF8091AF009091B000A0911C
:100BC000B100B091B200CD01AA27BB271DC0809112
:100BD000AF009091B000A091B100B091B200892F08
:100BE0009A2FAB2FBB2710C08091AF009091B0001F
:100BF000A091B100B091B20007C084B78F7083B9E3
:100C000014BE03C08091A30083B985EC11C080910C
:100C1000A60083B985EC86BF8091A00083B985ECDE
:100C200086BF80919F0083B985EC86BF13B885E8A5
:100C300086BF8091ED008F5F8093ED0004C085EC4E
:100C400001C085ED86BF80919F00823009F4A89590
:100C5000FF91EF91BF91AF919F918F917F916F9194
:100C60005F914F913F912F910F900FBE0F901F906A
:100C700018951F920F920FB60F9211242F933F9346
:100C80004F935F938F939F9389B380FF02C093E04C
:100C900001C090E081FF02C081E09827809193001D
:100CA000891B80FF1AC09093930090916900827015
:100CB0002091E2003091E300992329F090E0019720
:100CC000820F931F06C090E00197A901481B590BA2
:100CD000CA019093E3008093E20089B382958F70FC
:100CE00080FF02C093E001C090E081FF02C081E07C
:100CF000982780919200891B80FF1AC090939200E0
:100D00009091680082702091E0003091E100992379
:100D100039F090E00197A901481B590BCA0104C0A2
:100D200090E00197820F931F9093E1008093E00081
:100D300089B38695869580FF02C093E001C090E05C
:100D400081FF02C081E0982780919100891B80FF7C
:100D50001AC0909391009091D70082702091DE008C
:100D60003091DF00992339F090E00197A901481BE9
:100D7000590BCA0104C090E00197820F931F909312
:100D8000DF008093DE0089B3829586958695837017
:100D900080FF02C093E001C090E0827011F081E01A
:100DA000982780919000891B80FF1AC09093900033
:100DB0009091D60082702091DC003091DD00992363
:100DC00029F090E00197820F931F06C090E00197F1
:100DD000A901481B590BCA019093DD008093DC00E8
:100DE0008091C5008F5F8093C5009F918F915F9127
:100DF0004F913F912F910F900FBE0F901F9018951C
:100E00001F920F920FB60F9211242F933F934F937F
:100E10005F936F937F938F939F93AF93BF93EF9362
:100E2000FF938091C4008F5F8093C4009091C400B1
:100E30008091C300981778F01092C4008091E4006C
:100E40009091E5009195819591099093E5008093AB
:100E5000E4000E941501FF91EF91BF91AF919F9126
:100E60008F917F916F915F914F913F912F910F9053
:100E70000FBE0F901F9018951F920F920FB60F92F2
:100E800011248F939F93EF93FF935F9B16C0E09184
:100E9000F900F091FA008CB1808381E0EE35F8071B
:100EA00030F43196F093FA00E093F90006C08BEF2E
:100EB00090E09093FA008093F900FF91EF919F9159
:100EC0008F910F900FBE0F901F9018959C018AB1C3
:100ED00088618AB9579A80B5866080BDC901A0E053
:100EE000B0E09C01AD0184E0220F331F441F551F69
:100EF0008A95D1F760E47BE48CE490E00E943C1496
:100F0000DA01C9010197A109B109892F9A2FAB2FE5
:100F1000BB27A7FDBA9580BD215029B98BEF90E082
:100F20009093F8008093F7009093FA008093F90073
:100F300008955D9BFECFFC0180818CB90895CF930D
:100F4000DF931F92CDB7DEB78983CE0101960E9451
:100F5000990780E090E00F90DF91CF910895CF93B3
:100F6000DF93EC01CE012196FC012081222319F0B0
:100F70000E949907F7CFDF91CF9108955F9BFECF35
:100F80008CB190E008950C94BE0763EC77E08FE994
:100F900097E00C94C514CF93DF93FC01E253FF4F0D
:100FA000A081B181EC01C453DF4F28813981A217A0
:100FB000B307A1F05D9B12C02C912CB92081318127
:100FC000AC0145535F4F2417350718F42F5F3F4F8F
:100FD00003C09C0128593F4F31832083E091F700E3
:100FE000F091F8002091F9003091FA002E173F0798
:100FF000B1F1EC01CC59DF4FA881B98120812C934C
:10100000688179819C012B523F4FD9013C91DB01D2
:101010002C91321307C0AC014C525F4FDA012C9176
:101020002F5F2C939C012D593F4F6217730728F4B3
:10103000DB011196B983A88302C099838883B1E04C
:10104000EE35FB0730F43196F093F800E093F700AB
:1010500006C08BEF90E09093F8008093F700DF914B
:10106000CF910895CF93DF93CDB7DEB7A0970FB69A
:10107000F894DEBF0FBECDBF88E087BB8CEF84BB8A
:101080008CEB81BB87E088BB80E482BB1092EC00D4
:1010900080E895E20E9466070E94C50780E582B954
:1010A00085EC86BF81E08FBD89E08EBD1BBC1ABC7C
:1010B00019BC18BC89E485BD13BC83BF1CBE8AEC77
:1010C00091E09F938F930E944C1581E090E00E94E5
:1010D00014178093A00085B78F7885BF84E089BFFF
:1010E00078940F900F9022242A94312C00E010E87D
:1010F0008091ED00843A19F08F3F09F134C080915E
:101100009F00813061F428E13FE00FB6F894A89584
:1011100021BD0FBE31BD42E040939F0024C08091AD
:101120009F00811120C00FB6F894A89581B5886101
:1011300081BD11BC0FBE53E050939F0014C080913D
:10114000EC00853A81F4F8946BE780E090E00E942F
:101150001C17E199FECF88E198E00FB6F894A895A6
:1011600081BD0FBE91BD8091F600882309F4D9C0DE
:10117000F8948090EE009090EF00A090F000B09076
:10118000F1006091F2007091F3008091F400909171
:10119000F5001092F600789425E739E54CEC5EE313
:1011A0000E946A1320E030E040E05FE30E946A138F
:1011B000A50194010E9456116B017C01A5019401C7
:1011C000C501B4010E945611A70196010E94551154
:1011D00020E038E24EEA55E40E946A134B015C01BC
:1011E00020E038E24EEA55E4C701B6010E946A13D6
:1011F0006B017C018091A400882399F18091A40067
:1012000064E670E0681B7109072E000C880B990BCF
:101210000E947612A50194010E946A1320E030E03A
:1012200048EC52E40E94CC110E943E127093D5000B
:101230006093D4008091A40064E670E0681B71099B
:10124000072E000C880B990B0E947612A7019601BD
:101250000E946A1320E030E048EC52E40E94CC1176
:101260000AC0C501B4010E943E127093D50060937C
:10127000D400C701B6010E943E127093D100609362
:10128000D0008091A500882399F18091A50064E6A3
:1012900070E0681B7109072E000C880B990B0E94E7
:1012A0007612A50194010E946A1320E030E048EC18
:1012B00052E40E94CC110E943E127093D3006093BE
:1012C000D2008091A50064E670E0681B7109072ECA
:1012D000000C880B990B0E947612A70196010E94C0
:1012E0006A1320E030E048EC52E40E94CC110AC0BE
:1012F000C501B4010E943E127093D3006093D200E6
:10130000C701B6010E943E127093CF006093CE00D9
:1013100021E02093DB002093DA002093D900209372
:10132000D8008091C500833C08F49FC61092C50088
:10133000F8944091E2005091E3005A8349838091F0
:10134000E0009091E1009C838B832091DE0030913E
:10135000DF003E832D834091DC005091DD005887F3
:101360004F83789480918E0090918F00E980FA806D
:10137000E81AF90A80918C0090918D00CB80DC8076
:10138000C81AD90A80918A0090918B002901481AC5
:10139000590A80918800909189003A01681A790A67
:1013A000B7010F2C000C880B990B0E9476122AE0D3
:1013B00037ED43E25CE30E94CC110E943E126D8740
:1013C0007E878F87988BB6010D2C000C880B990BAC
:1013D0000E9476122AE037ED43E25CE30E94CC11D2
:1013E0000E943E12698B7A8B8B8B9C8BB201052CF1
:1013F000000C880B990B0E9476122AE037ED43E22D
:101400005CE30E94CC110E943E126D8B7E8B8F8B11
:10141000988FB301072C000C880B990B0E94761251
:101420002AE037ED43E25CE30E94CC110E943E12B9
:10143000698F7A8F8B8F9C8FB7016C0D7D1D072E66
:10144000000C880B990B0E94761220E038E24EE2E5
:1014500056E40E94CC114B015C01B201660D771D70
:10146000072E000C880B990B0E94761220E038E2C0
:101470004EE256E40E94CC112B013C01A5019401DF
:101480000E94551125E739E54CEC5EE30E94CC1132
:1014900069877A878B879C872091AF003091B00055
:1014A0004091B1005091B2000E9456116B017C0135
:1014B0002BED3FE049EC50E40E94651318164CF404
:1014C0002BED3FE049EC50E4C701B6010E945511F5
:1014D00012C02BED3FE049EC50ECC701B6010E9471
:1014E000C21187FF0AC02BED3FE049EC50E4C70171
:1014F000B6010E9456116B017C01A3019201C50146
:10150000B4010E94561120E030E040E05FE30E9409
:101510006A134B015C014090B7005090B800609096
:10152000B9007090BA00C701B6010E94C7119B01B3
:10153000AC01C501B4010E946A13A30192010E948B
:1015400056116D8F7E8F8F8F98A34090B30050906F
:10155000B4006090B5007090B600C701B6010E945B
:10156000D7139B01AC01C501B4010E946A13A3010A
:1015700092010E9456112B013C012AE037ED43E213
:101580005CE3C501B4010E94CC114B015C012AE06F
:1015900037ED43E25CE369857A858B859C850E9403
:1015A000CC11F894C092AF00D092B000E092B1009C
:1015B000F092B2002D8D3E8D4F8D58A12093B70033
:1015C0003093B8004093B9005093BA004092B300F2
:1015D0005092B4006092B5007092B6004D855E8561
:1015E0005093C2004093C10029893A893093C000CA
:1015F0002093BF004D895E895093BE004093BD008B
:10160000298D3A8D3093BC002093BB008092AB00B3
:101610009092AC00A092AD00B092AE006093A70093
:101620007093A8008093A9009093AA0078944981B0
:101630005A8150938F0040938E008B819C819093B0
:101640008D0080938C002D813E8130938B00209300
:101650008A004F815885509389004093880080917B
:10166000840090918500A0918600B0918700B7FF1B
:1016700007C0B095A095909581959F4FAF4FBF4FF4
:10168000813E9242A240B105CCF08091C100909180
:10169000C200892B99F41092EB001092EA0010928C
:1016A000DB008091A30080618093A30010928400EE
:1016B0001092850010928600109287008091800021
:1016C00090918100A0918200B0918300B7FF07C084
:1016D000B095A095909581959F4FAF4FBF4F813E9C
:1016E0009242A240B105CCF08091BF009091C00021
:1016F000892B99F41092E9001092E8001092DA0018
:101700008091A30080628093A300109280001092C9
:101710008100109282001092830080917C00909151
:101720007D00A0917E00B0917F00B7FF07C0B0950B
:10173000A095909581959F4FAF4FBF4F813E9242AC
:10174000A240B105CCF08091BD009091BE00892BE4
:1017500099F41092E7001092E6001092D90080915F
:10176000A30080648093A30010927C0010927D00FF
:1017700010927E0010927F00809178009091790005
:10178000A0917A00B0917B00B7FF07C0B095A095FB
:10179000909581959F4FAF4FBF4F813E9242A2409F
:1017A000B105CCF08091BB009091BC00892B99F4DD
:1017B0001092E5001092E4001092D8008091A300EE
:1017C00080688093A30010927800109279001092A4
:1017D0007A0010927B008091DB00813009F0FCC020
:1017E0002091D4003091D5008091CC009091CD0013
:1017F0002817390711F18091D4009091D5002091DC
:10180000CC003091CD00821B930B97FF03C09195C4
:1018100081959109853F914044F010928400109287
:10182000850010928600109287008091D4009091DC
:10183000D5009093CD008093CC008091D4009091FE
:10184000D5001816190634F48091C1009091C20099
:1018500097FD0FC08091D4009091D50097FF0BC0E9
:101860008091C1009091C20021E01816190624F061
:1018700002C021E001C020E08091D4009091D50009
:10188000892B11F0222371F01092EB001092EA00E4
:1018900010927700109276008091A3008F7E809343
:1018A000A3009AC0E090D400F090D5008091C100D0
:1018B0009091C200E81AF90AB7010F2C000C880BAE
:1018C000990B8090840090908500A0908600B09045
:1018D0008700860E971EA81EB91E809284009092E3
:1018E0008500A0928600B09287000E94761226EBB7
:1018F00033EF4DE75DE30E946A132B013C01C50104
:10190000B4010E94761221E539E44DE95AE30E94C0
:101910006A139B01AC01C301B2010E9456114B0135
:101920005C018091760090917700B701681B790B7C
:10193000072E000C880B990B0E94761220E030E0F5
:10194000A9010E946A139B01AC01C501B4010E9468
:1019500056110E943E127093EB006093EA00F092E1
:101960007700E09276008091EA009091EB001816E3
:10197000190634F48091D4009091D50097FD0DC0E4
:101980008091EA009091EB0097FF0CC08091D40009
:101990009091D500181619062CF41093EB000093C3
:1019A000EA001AC08091EA009091EB008F3F910508
:1019B00031F02CF03092EB002092EA000DC08091C3
:1019C000EA009091EB0081309F4F34F441E05FEFEB
:1019D0005093EB004093EA008091DA00813009F0E7
:1019E000FCC02091D2003091D3008091CA00909128
:1019F000CB002817390711F18091D2009091D300C4
:101A00002091CA003091CB00821B930B97FF03C03B
:101A1000919581959109853F914044F01092800005
:101A20001092810010928200109283008091D20067
:101A30009091D3009093CB008093CA008091D20004
:101A40009091D3001816190634F48091BF0090913C
:101A5000C00097FD0FC08091D2009091D30097FFF6
:101A60000BC08091BF009091C00021E018161906AC
:101A700024F002C021E001C020E08091D2009091CA
:101A8000D300892B11F0222371F01092E9001092FB
:101A9000E80010927500109274008091A3008F7D71
:101AA0008093A3009AC0E090D200F090D300809180
:101AB000BF009091C000E81AF90AB7010F2C000C82
:101AC000880B990B8090800090908100A0908200FC
:101AD000B0908300860E971EA81EB91E80928000CB
:101AE00090928100A0928200B09283000E947612B0
:101AF00026EB33EF4DE75DE30E946A132B013C01B7
:101B0000C501B4010E94761221E539E44DE95AE39A
:101B10000E946A139B01AC01C301B2010E945611DD
:101B20004B015C018091740090917500B701681BB6
:101B3000790B072E000C880B990B0E94761220E07F
:101B400030E0A9010E946A139B01AC01C501B401F8
:101B50000E9456110E943E127093E9006093E800C3
:101B6000F0927500E09274008091E8009091E90095
:101B70001816190634F48091D2009091D30097FD85
:101B80000DC08091E8009091E90097FF0CC0809112
:101B9000D2009091D300181619062CF41093E90086
:101BA0000093E8001AC08091E8009091E9008F3F0F
:101BB000910531F02CF03092E9002092E8000DC040
:101BC0008091E8009091E90081309F4F34F441E02A
:101BD0005FEF5093E9004093E8008091D900813095
:101BE00009F0FCC02091D0003091D1008091C80054
:101BF0009091C9002817390711F18091D000909178
:101C0000D1002091C8003091C900821B930B97FF2F
:101C100003C0919581959109853F914044F01092C0
:101C20007C0010927D0010927E0010927F008091C7
:101C3000D0009091D1009093C9008093C80080910A
:101C4000D0009091D1001816190634F48091BD008F
:101C50009091BE0097FD0FC08091D0009091D1006F
:101C600097FF0BC08091BD009091BE0021E0181637
:101C7000190624F002C021E001C020E08091D000CC
:101C80009091D100892B11F0222371F01092E7007E
:101C90001092E60010927300109272008091A300DF
:101CA0008F7B8093A3009AC0E090D000F090D10089
:101CB0008091BD009091BE00E81AF90AB7010F2C7F
:101CC000000C880B990B80907C0090907D00A09078
:101CD0007E00B0907F00860E971EA81EB91E8092CF
:101CE0007C0090927D00A0927E00B0927F000E94C6
:101CF000761226EB33EF4DE75DE30E946A132B016A
:101D00003C01C501B4010E94761221E539E44DE998
:101D10005AE30E946A139B01AC01C301B2010E9405
:101D200056114B015C018091720090917300B701D4
:101D3000681B790B072E000C880B990B0E947612FA
:101D400020E030E0A9010E946A139B01AC01C501AB
:101D5000B4010E9456110E943E127093E7006093F6
:101D6000E600F0927300E09272008091E60090919C
:101D7000E7001816190634F48091D0009091D10034
:101D800097FD0DC08091E6009091E70097FF0CC091
:101D90008091D0009091D100181619062CF4109360
:101DA000E7000093E6001AC08091E6009091E700FA
:101DB0008F3F910531F02CF03092E7002092E60041
:101DC0000DC08091E6009091E70081309F4F34F480
:101DD00041E05FEF5093E7004093E6008091D80028
:101DE000813009F0FCC02091CE003091CF0080916D
:101DF000C6009091C7002817390711F18091CE00D5
:101E00009091CF002091C6003091C700821B930BA8
:101E100097FF03C0919581959109853F914044F0CA
:101E2000109278001092790010927A0010927B0044
:101E30008091CE009091CF009093C7008093C60010
:101E40008091CE009091CF001816190634F480913D
:101E5000BB009091BC0097FD0FC08091CE00909187
:101E6000CF0097FF0BC08091BB009091BC0021E098
:101E70001816190624F002C021E001C020E080916C
:101E8000CE009091CF00892B11F0222371F0109297
:101E9000E5001092E40010927100109270008091A1
:101EA000A3008F778093A3009AC0E090CE00F090BB
:101EB000CF008091BB009091BC00E81AF90AB701ED
:101EC0000F2C000C880B990B809078009090790073
:101ED000A0907A00B0907B00860E971EA81EB91EB7
:101EE0008092780090927900A0927A00B0927B0064
:101EF0000E94761226EB33EF4DE75DE30E946A13F2
:101F00002B013C01C501B4010E94761221E539E4A0
:101F10004DE95AE30E946A139B01AC01C301B2016F
:101F20000E9456114B015C018091700090917100EC
:101F3000B701681B790B072E000C880B990B0E94C8
:101F4000761220E030E0A9010E946A139B01AC01E7
:101F5000C501B4010E9456110E943E127093E50023
:101F60006093E400F0927100E09270008091E400D0
:101F70009091E5001816190634F48091CE009091E6
:101F8000CF0097FD0DC08091E4009091E50097FF90
:101F90000CC08091CE009091CF00181619062CF439
:101FA0001093E5000093E4001AC08091E400909142
:101FB000E5008F3F910531F02CF03092E500209242
:101FC000E4000DC08091E4009091E50081309F4FC6
:101FD00034F441E05FEF5093E5004093E4000E9449
:101FE00015018091A6008F5F8093A6008091A200CA
:101FF0008F3FD9F18091A2008F5F8093A2008091E2
:10200000A200843690F11092EE001092EF00109230
:10201000F0001092F1001092F2001092F300109272
:10202000F4001092F50051E05093F6008091A20068
:10203000843621F08FEF8093A20017C08091A10019
:102040001F928F9328EB31E03F932F930E944C1502
:102050006091A10081E090E00E941C170F900F900A
:102060000F900F90E199FECFE5CF85B7806885BFCF
:10207000889585B78F7785BF3BC8ABE0B0E0E3E4D8
:10208000F0E10C9465146C017B013A01FC011782AC
:102090001682838181FF03C1CE0101964C01F601B6
:1020A000B380F701B3FC0591B3FE01917F010023DA
:1020B00009F4F1C0053249F4B3FC0591B3FE019176
:1020C0007F01053211F010E019C0B601802F90E0B9
:1020D0000E94101553013501E2CF002309F4DBC043
:1020E000602F70E08BED91E00E94BA14892B49F0CB
:1020F000F701B3FC0591B3FE01917F0117FFEDCF0E
:1021000004C0033239F00C3619F0011105C0C3C008
:102110001068EECF10E1ECCF602F70E084ED91E01D
:102120000E94BA14892B41F05301F4E0AF0EB11CA8
:10213000B6018FE390E010C0033631F0033779F039
:10214000033511F511600BC0530182E0A80EB11CDC
:10215000B601F301808191810E941015BCCF53011B
:10216000F2E0AF0EB11CF30160807180F30110FD4D
:10217000859110FF81913F01882309F4ACCFB6010E
:1021800090E00E941015F2CF043611F0093621F5C7
:10219000530117FF09C0F4E0AF0EB11CF3016081D9
:1021A0007181828193810AC0F2E0AF0EB11CF3010C
:1021B00060817181072E000C880B990B1F7E97FFA1
:1021C00008C090958095709561957F4F8F4F9F4F78
:1021D00010642AE030E030C0003791F040F4083558
:1021E000A1F00F3609F057C028E030E011C00537E4
:1021F00019F0083731F04FC01F7E2AE030E008C0E8
:102200001061146220E130E003C0146020E132E08C
:10221000530117FF09C0F4E0AF0EB11CF301608158
:1022200071818281938108C0F2E0AF0EB11CF3018D
:102230006081718180E090E0A4010E947215082FF6
:10224000081916FF05C0B6018DE290E00E94101536
:1022500014FF15C0FE01E00FF11D8081803379F07D
:10226000B60180E390E00E94101512FF08C01072C2
:10227000812F90E0B601885A9F4F0E94101501509F
:10228000F401E00FF11D8081B60190E00E9410156D
:102290000111F5CF20CFF6018681978102C08FEF23
:1022A0009FEF2B96EEE00C9481145058BB27AA2781
:1022B0000E946D110C9417130E94DE1238F00E94D8
:1022C000E51220F039F49F3F19F426F40C94DB1248
:1022D0000EF4E095E7FB0C94D512E92F0E943C1315
:1022E00058F3BA17620773078407950720F079F44B
:1022F000A6F50C945E130EF4E0950B2EBA2FA02DCC
:102300000B01B90190010C01CA01A0011124FF27A2
:10231000591B99F0593F50F4503E68F11A16F0409D
:10232000A22F232F342F4427585FF3CF469537959C
:102330002795A795F0405395C9F77EF41F16BA0B61
:10234000620B730B840BBAF09150A1F0FF0FBB1F0F
:10235000661F771F881FC2F70EC0BA0F621F731F58
:10236000841F48F4879577956795B795F7959E3FB5
:1023700008F0B0CF9395880F08F09927EE0F979546
:10238000879508950E94B11208F481E008950E9493
:10239000EE12E3950C9428130E94E0110C9417138D
:1023A0000E94E51258F00E94DE1240F029F45F3FCF
:1023B00029F00C94D51251110C945F130C94DB127C
:1023C0000E943C1368F39923B1F3552391F3951BB5
:1023D000550BBB27AA2762177307840738F09F5F46
:1023E0005F4F220F331F441FAA1FA9F335D00E2EB3
:1023F0003AF0E0E832D091505040E695001CCAF720
:102400002BD0FE2F29D0660F771F881FBB1F2617E2
:1024100037074807AB07B0E809F0BB0B802DBF01B9
:10242000FF2793585F4F3AF09E3F510578F00C9488
:10243000D5120C945F135F3FE4F3983ED4F3869576
:1024400077956795B795F7959F5FC9F7880F911DA9
:102450009695879597F90895E1E0660F771F881F95
:10246000BB1F621773078407BA0720F0621B730B48
:10247000840BBA0BEE1F88F7E09508950E94451271
:102480006894B1110C945F1308950E94441388F06E
:102490009F5798F0B92F9927B751B0F0E1F0660F28
:1024A000771F881F991F1AF0BA95C9F714C0B13069
:1024B00091F00E945E13B1E008950C945E13672FB3
:1024C000782F8827B85F39F0B93FCCF38695779598
:1024D0006795B395D9F73EF4909580957095619581
:1024E0007F4F8F4F9F4F0895E89409C097FB3EF4AC
:1024F00090958095709561957F4F8F4F9F4F992351
:10250000A9F0F92F96E9BB279395F69587957795CE
:102510006795B795F111F8CFFAF4BB0F11F460FF8E
:102520001BC06F5F7F4F8F4F9F4F16C0882311F0E6
:1025300096E911C0772321F09EE8872F762F05C0FA
:10254000662371F096E8862F70E060E02AF09A9595
:10255000660F771F881FDAF7880F9695879597F98A
:102560000895990F0008550FAA0BE0E8FEEF161624
:102570001706E807F907C0F012161306E407F50777
:1025800098F0621B730B840B950B39F40A2661F0EB
:10259000232B242B252B21F408950A2609F4A1408E
:1025A000A6958FEF811D811D089597F99F6780E89B
:1025B00070E060E008959FEF80EC089500240A9495
:1025C0001616170618060906089500240A9412160E
:1025D00013061406050608950C94DB120E9444139A
:1025E000D8F3E894E0E0BB279F57F0F02AED3FE0F6
:1025F00049EC06C0EE0FBB0F661F771F881F28F03F
:10260000B23A62077307840728F0B25A620B730B61
:10261000840BE3959A9572F7803830F49A95BB0F46
:10262000661F771F881FD2F790480C94E113092E7C
:102630000394000C11F4882352F0BB0F40F4BF2B1D
:1026400011F460FF04C06F5F7F4F8F4F9F4F08955D
:10265000EF93E0FF07C0A2EA2AED3FE049EC5FEB11
:102660000E946D110E9417130F90039401FC905863
:10267000EAE9F1E00C94ED1357FD9058440F551F13
:1026800059F05F3F71F04795880F97FB991F61F0F4
:102690009F3F79F087950895121613061406551F6B
:1026A000F2CF4695F1DF08C0161617061806991FD7
:1026B000F1CF86957105610508940895E894BB27CC
:1026C00066277727CB0197F908950E94B11208F485
:1026D0008FEF08950E947D130C9417130E94DE1251
:1026E00038F00E94E51220F0952311F00C94D512D9
:1026F0000C94DB1211240C945F130E943C1370F3B2
:10270000959FC1F3950F50E0551F629FF001729F96
:10271000BB27F00DB11D639FAA27F00DB11DAA1FA5
:10272000649F6627B00DA11D661F829F2227B00DF2
:10273000A11D621F739FB00DA11D621F839FA00D7D
:10274000611D221F749F3327A00D611D231F849FCD
:10275000600D211D822F762F6A2F11249F57504024
:102760009AF0F1F088234AF0EE0FFF1FBB1F661F9F
:10277000771F881F91505040A9F79E3F510580F068
:102780000C94D5120C945F135F3FE4F3983ED4F39E
:10279000869577956795B795F795E7959F5FC1F70C
:1027A000FE2B880F911D9695879597F908959F9315
:1027B0000E94EE120F9007FCEE5F0C9428139F3FCF
:1027C00031F0915020F4879577956795B795880FEC
:1027D000911D9695879597F908959F938F937F9371
:1027E0006F93FF93EF939B01AC010E946A13EF91EB
:1027F000FF910E9401142F913F914F915F910C9492
:102800006A13DF93CF931F930F93FF92EF92DF92A0
:102810007B018C01689406C0DA2EEF010E947D13C3
:10282000FE01E894A5912591359145915591A6F326
:10283000EF010E946D11FE019701A801DA9469F77A
:10284000DF90EF90FF900F911F91CF91DF9108954E
:10285000AA1BBB1B51E107C0AA1FBB1FA617B707C6
:1028600010F0A61BB70B881F991F5A95A9F78095E2
:102870009095BC01CD010895052E97FB1EF40094A0
:102880000E94531457FD07D00E94981407FC03D0F0
:102890004EF40C94531450954095309521953F4F2C
:1028A0004F4F5F4F089590958095709561957F4F3C
:1028B0008F4F9F4F0895EE0FFF1F0590F491E02D6D
:1028C00009942F923F924F925F926F927F928F92D4
:1028D0009F92AF92BF92CF92DF92EF92FF920F93AF
:1028E0001F93CF93DF93CDB7DEB7CA1BDB0B0FB6B9
:1028F000F894DEBF0FBECDBF09942A883988488876
:102900005F846E847D848C849B84AA84B984C8840B
:10291000DF80EE80FD800C811B81AA81B981CE0F02
:10292000D11D0FB6F894DEBF0FBECDBFED010895E7
:10293000A1E21A2EAA1BBB1BFD010DC0AA1FBB1FC3
:10294000EE1FFF1FA217B307E407F50720F0A21B35
:10295000B30BE40BF50B661F771F881F991F1A94A2
:1029600069F760957095809590959B01AC01BD01CC
:10297000CF010895FC010590061621F00020D9F73B
:10298000C00108953197CF0108950F931F93CF93FE
:10299000DF93009731F46115710519F480E090E040
:1029A0003AC08B01EC016EE070E081E090E00E94A3
:1029B000D015FC01892B91F380E883830115110563
:1029C00071F01387028781E883838091620190917F
:1029D0006301892B21F4F0936301E0936201209756
:1029E000C9F0D187C087838182608383809164012D
:1029F00090916501892B71F4F0936501E093640176
:102A00008091660190916701892B21F4F093670111
:102A1000E0936601CF01DF91CF911F910F9108954F
:102A20000F931F93CF93DF93FB01238121FD03C0FD
:102A30008FEF9FEF2CC022FF16C046815781248163
:102A400035814217530744F4A081B1819D012F5F66
:102A50003F4F318320838C93268137812F5F3F4FF7
:102A60003783268314C08B01EC01FB010084F185C0
:102A7000E02D0995892BE1F6D80116968D919C9150
:102A80001797019617969C938E931697CE01DF9118
:102A9000CF911F910F910895A0E0B0E0E2E5F5E13C
:102AA0000C946F14AE01495F5F4FDA016D917D9117
:102AB000AD0102E611E0F80182819381DC011396F9
:102AC0002C911397286013962C930E943D10D801E7
:102AD0001296ED91FC9113972381277F2383E4E0E5
:102AE0000C948B14FA01AA27283051F1203181F17E
:102AF000E8946F936E7F6E5F7F4F8F4F9F4FAF4F06
:102B0000B1E03ED0B4E03CD0670F781F891F9A1F18
:102B1000A11D680F791F8A1F911DA11D6A0F711DCC
:102B2000811D911DA11D20D009F468943F912AE0D8
:102B3000269F11243019305D3193DEF6CF010895C0
:102B4000462F4770405D4193B3E00FD0C9F7F6CFF1
:102B5000462F4F70405D4A3318F0495D31FD4052B9
:102B6000419302D0A9F7EACFB4E0A695979587954F
:102B700077956795BA95C9F700976105710508952E
:102B80009B01AC010A2E06945795479537952795DA
:102B9000BA95C9F7620F731F841F951FA01D089572
:102BA0000F931F93CF93DF93869F8001879F100D14
:102BB000969F100D1124C8010E94EC15EC0100979E
:102BC00029F0A80160E070E00E940D17CE01DF91AE
:102BD000CF911F910F9108950F931F93CF93DF9380
:102BE0008230910510F482E090E0E0916A01F0916A
:102BF0006B0120E030E0A0E0B0E0309719F14081B7
:102C000051810281138148175907C8F0841795072D
:102C100069F4109731F012960C93129713961C9347
:102C200027C000936A0110936B0122C02115310562
:102C300019F04217530718F49A01BD01EF01DF01A3
:102C4000F801DBCF21153105F9F0281B390B2430B1
:102C5000310580F48A819B816115710521F0FB01AA
:102C60009383828304C090936B0180936A01FE0179
:102C7000329644C0FE01E20FF31F819391932250DC
:102C80003109398328833AC0209168013091690164
:102C9000232B41F420916C0030916D003093690139
:102CA0002093680120916A0030916B002115310555
:102CB00041F42DB73EB740916E0050916F00241B38
:102CC000350BE0916801F0916901E217F307A0F478
:102CD0002E1B3F0B2817390778F0AC014E5F5F4F72
:102CE0002417350748F04E0F5F1F5093690140933A
:102CF00068018193919302C0E0E0F0E0CF01DF91A1
:102D0000CF911F910F910895CF93DF93009709F40E
:102D100081C0FC01329713821282A0916A01B091A6
:102D20006B01109781F420813181820F931F2091D4
:102D30006801309169012817390751F5F09369014D
:102D4000E093680167C0ED0120E030E0CE17DF07B7
:102D500040F44A815B819E0141155105F1F0EA0181
:102D6000F5CFD383C28340815181840F951FC8174B
:102D7000D90759F488819981840F951F0296918310
:102D800080838A819B81938382832115310529F475
:102D9000F0936B01E0936A013DC0E901FB83EA8394
:102DA00049915991C40FD51FEC17FD0761F480813B
:102DB0009181840F951F0296E9019983888382810E
:102DC00093819B838A83E0E0F0E012968D919C9141
:102DD0001397009719F0FD01DC01F7CF8D919C91BD
:102DE00011979D012E5F3F4F820F931F2091680125
:102DF000309169012817390769F4309729F4109246
:102E00006B0110926A0102C013821282B0936901B1
:102E1000A0936801DF91CF910895DC0101C06D930B
:102E200041505040E0F70895E199FECF9FBB8EBB23
:102E3000E09A99278DB30895262FE199FECF9FBB85
:102E40008EBB2DBB0FB6F894E29AE19A0FBE0196A5
:062E50000895F894FFCF85
:102E56000080008000800080010100006C012000DD
:00000001FF
